:020000000528D1
:100008000900831614308500CE3090008312073023
:10001800990005104E30982045309820543098208B
:100028000D3098200514051A1C28051D21281728AD
:100038000510AE203020051417284F2005109820F1
:10004800051417283C3098204A3098203E309820D4
:100058004F2020182C280E28A30002308420831655
:100068000511831204304720023047200830A600CB
:100078000130A30D031803304720A60B3C28831634
:10008800051583120800A2008B2005118B20A20BF6
:100098004A28051508002010A01005190800672037
:1000A8006720A1000830A600A3016720031965286E
:1000B800A2002108A202A30DA60B59282308A01408
:1000C800080020140800A201A20A03190800000071
:1000D80000000000000000000000000000000519FA
:1000E8006828A201A20A0319080000000000000005
:1000F80000000000000000002208051D7628080006
:10010800A5008D20A50B8528080001308E280A300F
:100118008E286430A40000000000000000000000E9
:100128000000A40B8F280800A200A601A6158512BE
:1001380000000000000000000000C220A20C031C08
:10014800851203188516A60BA028C2208516C22082
:10015800C2200800A601A615A201051EB128C420C8
:10016800051EAE28C2200310051E0314A20C0000B1
:100178000000A60BB628C220220808000C30C528AB
:100188000630AB00AB0BC6280800A900A800A80BD6
:08019800CB28A90BCA280800BE
:02400E00A4010B
:00000001FF
